:020000040800F2
:10000000A80B0020B902000821260008C924000816
:1000100019260008A9100008E130000800000000BF
:10002000000000000000000000000000612E000839
:10003000C110000800000000312B0008013000084A
:10004000D3020008D3020008D3020008D30200083C
:10005000D3020008D3020008D3020008D30200082C
:10006000D3020008D3020008D3020008D30200081C
:10007000D3020008D3020008D3020008B110000820
:10008000D3020008D3020008D3020008D3020008FC
:10009000D3020008D3020008D3020008D3020008EC
:1000A000D3020008D3020008D3020008D3020008DC
:1000B000D3020008D3020008D3020008D3020008CC
:1000C000D3020008D3020008D3020008D3020008BC
:1000D000392B0008D3020008D3020008D30200081D
:1000E000D3020008D3020008D3020008D30200089C
:1000F000D3020008D3020008D3020008D30200088C
:10010000D3020008D3020008D3020008D30200087B
:10011000D3020008D3020008D3020008D30200086B
:10012000D3020008D3020008D3020008D30200085B
:10013000D3020008D3020008D3020008D30200084B
:10014000D3020008D3020008D3020008D30200083B
:10015000D3020008D3020008D3020008D30200082B
:10016000D3020008D3020008D3020008D30200081B
:10017000D3020008D3020008D302000800000000E8
:10018000D3020008D3020008D3020008D3020008FB
:10019000D3020008D3020008D3020008D3020008EB
:1001A000D3020008D3020008D3020008D3020008DB
:1001B000D3020008D3020008D3020008D3020008CB
:1001C000D3020008D302000800F002F800F04BF858
:1001D0000AA090E8000C82448344AAF10107DA45A2
:1001E00001D100F040F8AFF2090EBAE80F0013F0A9
:1001F000010F18BFFB1A43F00103184764320000D7
:1002000084320000103A24BF78C878C1FAD8520767
:1002100024BF30C830C144BF04680C607047000080
:100220000023002400250026103A28BF78C1FBD8FF
:10023000520728BF30C148BF0B607047642900F0E7
:100240001381002070471FB503F0E2F89DE803001A
:1002500000F01AFD00F059F900F052FA1FBD10B578
:1002600000F0B7FA10BD00F0E7FA1146FFF7EBFF18
:1002700002F0BEFF00F0D8FC03B4FFF7F0FF03BCB0
:1002800000F07CFE0B49D1F800C04A685CF8043BE2
:100290001068184442F8040B8C4528BFA1F1DC0C0F
:1002A0008A4228BFA1F1DC02C1F800C04A6020F0F8
:1002B00000407047FC00002009488047094800477B
:1002C000FEE7FEE7FEE7FEE7FEE7FEE7FEE7FEE706
:1002D000FEE7FEE704480549054A064B7047000063
:1002E000C9300008C9010008A8050020A80B00209B
:1002F000A8070020A807002053EA020C00F069803C
:100300002DE9F04B4FF00006002B1FBFB3FA83F529
:1003100003FA05F424FA05F65E4012BF1643B2FA5A
:1003200082F502FA05F4C5F120051EBF22FA05FC8C
:1003300044EA0C04203556EA044C4FEA144418BF32
:10034000641C4FF000084FF00009904271EB030C61
:1003500039D3002919BFB1FA81F701FA07F6B0FACB
:1003600080F700FA07F6C7F120071EBF20FA07FC46
:1003700046EA0C062037B6FBF4FCA7EB0507103F56
:1003800007F01F0BCBF120062CFA06F60CFA0BFB3C
:1003900044BFB3460026202FA4BF5E464FF0000B9B
:1003A0005BEA060C08BF4FF0010B19EB0B0948EB99
:1003B0000608ABFB027C06FB02CC0BFB03CCC01B8C
:1003C00071EB0C01C1E70B46024641464846BDE8C9
:1003D000F08B13B5084318BF4FF0FF300146AFF361
:1003E0000080BDE81C4070470FB4044910B503AA53
:1003F000029800F02FF910BC5DF814FB58010020A2
:100400002DE9F0410E460446002020622046E168B6
:10041000884730B3252805D0D4E901219047206AC8
:10042000401CF2E7E168204600278847050018D005
:10043000A5F14100192802D820354FF40067324653
:10044000294620462760FFF7F9FE40B1012804D075
:10045000F61D26F007060836D8E7361DD6E72846EB
:10046000DAE7206ABDE8F0812DE9F0410646002474
:1004700010687529314616A510D0AFF3008000280A
:1004800002DA404213A507E031688A0701D512A5B8
:1004900002E0490704D511A5012401E0AFF3008073
:1004A00000210A2206F1240709E0B0FBF2FCB0FBB0
:1004B000F2F302FB1C00303078541846491C002827
:1004C000F3D123462A463046BDE8F04100F069B832
:1004D000000000002D0000002B00000020000000A4
:1004E0000B4910B5A1F17C020A4CC2E93712372141
:1004F00006E000EB104342F82130074B00FB0340BD
:100500000B1EA1F10101F4DC10BD0120E8E70000A1
:100510009C000020E119D666CD0D0100000000000E
:1005200030B44FF0013C50F8042BCCFA52F451F89F
:10053000043BD51A20D1FCB950F8042BCCFA52F464
:1005400051F8043BD51A17D1B4B950F8042BCCFAA2
:1005500052F451F8043BD51A0ED16CB950F8042B63
:10056000CCFA52F451F8043BD51A05D1002CDAD05C
:1005700030BC4FF00000704729BAB1FA81F111F098
:100580001801D1F120008440F2D1CA40CB4012F0D2
:10059000FF0213F0FF0330BCD01A7047704770475A
:1005A00070472DE9F0470D4699469246044600F102
:1005B00024080168880604D5E06921F01001216053
:1005C00000E00120A84201DD471B00E00027A169EF
:1005D0007A1902EB0900081AA0612078C00602D43B
:1005E0002046AFF30080002608E0D4E901211AF884
:1005F00006009047206A401C761C20624E45F4DBC2
:100600002078C0060AD52046AFF3008006E0D4E982
:10061000012130209047206A401C2062381EA7F13B
:100620000107F4DC07E0D4E9012118F80500904740
:10063000206A401C2062281EA5F10105F3DC20463B
:10064000AFF300802078000602D50220BDE8F087D5
:100650000120FBE7074B70B50D467B4400F039F8ED
:100660000446284600F048F810B14FF0FF3070BD46
:10067000204670BD992D00004FF0000200B51346D2
:1006800094469646203922BFA0E80C50A0E80C50B2
:10069000B1F12001BFF4F7AF090728BFA0E80C5063
:1006A00048BF0CC05DF804EB890028BF40F8042B5C
:1006B00008BF704748BF20F8022B11F0804F18BFC9
:1006C00000F8012B7047000001694A1C026108789C
:1006D000704700B58FB0CDE9013100210591054982
:1006E0007944CDE9031011466846FFF789FE0FB043
:1006F00000BD0000E5FFFFFF007B00F080007047B9
:1007000010B542485421FFF7B7FF41485421FFF785
:10071000B3FF40485421FFF7AFFF3F493B483C4AF5
:100720003F4B08603D490A603A491960531C036514
:10073000481C1065012008653B48344A39A17844BB
:1007400000F0D4F920B9384878440A3800F075FA36
:1007500037482F4A35A1784400F0C8F920B9344809
:1007600078440A3800F069FA32482A4A2FA17844BE
:1007700000F0BCF920B92F4878440A3800F05DFA3F
:1007800040232248DC000021224600F08CF920B1F1
:1007900025487844543800F050FA1D48224640233A
:1007A000002100F080F920B121487844543800F04D
:1007B00044FA184822461023002100F074F900285A
:1007C00006D01C487844BDE81040563800F035BAD1
:1007D00010BD104870B5006D20F001040B4800F00A
:1007E000FDF90B4800F0FAF90A4800F0F7F909E0C2
:1007F000206D20F00105204600F0F0F9204600F0C1
:1008000040F82C46002CF3D170BD000004010020FC
:1008100058010020AC01002000000020040000204E
:100820000800002072000000002D0000770000008A
:10083000EF2C0000C82C0000754600F005FAAE460B
:1008400005006946534620F00700854618B020B5DC
:10085000FFF740FDBDE820404FF000064FF00007D5
:100860004FF000084FF0000BAC46ACE8C009ACE814
:10087000C009ACE8C009ACE8C00921F007018D4609
:10088000704770B50446051F00F0E2F90068002CBF
:1008900014BF446870BD002C18BFAC423CBF20465A
:1008A0006468F8D301680A18AA4218BF456003D1EA
:1008B0002A6805461144016028684119A1421CBFFD
:1008C0006C6070BD6168696021680844286070BD13
:1008D0002DE9F04705460C46C86820F4201040F486
:1008E0008000C860800602D5084600F0FEFAE06885
:1008F00041F282014FF0FF390140022903D0204626
:1009000000F09CFAB5E000F42041B1F5004F0FD1A2
:10091000C00306D56168E06A884200D80846606076
:1009200006E02069E0626060606902F0E9FBA061B6
:10093000A0680022EEB200280DDAE1688B050AD427
:10094000C043A06041F490302260E0606068411CC8
:1009500061600670A5E0E0689046226040F40050B7
:10096000E060206968BB606902F0CEFB012704F1FA
:100970002405A0B1A08910F4407F08D0E06900F000
:10098000B2F9206118B1E06840F4006016E0E76158
:100990002561E06820F4407040F480600EE0E0697A
:1009A00000F0A1F900282061F1D0E06840F4006077
:1009B00010F4407FE06002D140F48070E060206974
:1009C0006060E06825696FF0010AC1051FD56168A4
:1009D000E06A884200D80846411B04D022462846D7
:1009E00000F036FAF0BBE068010203D5E562C4E925
:1009F000015854E0691CE1626160E16940F48030B3
:100A0000491EC4E9021030462E70BDE8F08701028D
:100A100002D500F480320AE06068411C6160067013
:100A2000E0680A2E40F48030E06006D00022E16ADF
:100A30006068814203D90B4602E00122F7E70346D2
:100A4000A7895B1B7F0503D4E7699F4200DDE2B104
:100A5000814200D80146E5620F1AC4E90158002B13
:100A600009DD00E005E022461946284600F0F0F9CD
:100A700008B14846C9E747B1A069E5626560C01B97
:100A8000A061E06840F01000E060E068000208D576
:100A90006168A069E562491B08446560A061504631
:100AA000B3E73046B1E770B5C468A50713D0650257
:100AB00011D4B2F5807F09D0B2F5007F06D0B2F52F
:100AC000806F08D1012300F1240106E05D1E6FF064
:100AD0007F46B54201D3012070BD0161C361416011
:100AE00024F470611143C160002070BD2DE9F04114
:100AF0000C461646070047D0104600F06FF82078E5
:100B0000611C61280AD0722802D077283CD102E00B
:100B10000125002405E00225042402E0082448F20F
:100B2000020511F8010B2B2806D0622809D011F814
:100B3000010C74280AD00BE045F0030544F00204D0
:100B4000EFE745F0040544F00104EAE744F010043F
:100B50003846214602F0E0FA411C15D000213161EF
:100B600071604FF40071F560F1617061200704D588
:100B700030460222002100F0E5F8306D40F001001F
:100B800030653046BDE8F0810020FBE72DE9F041FB
:100B90000D460646104C206DC10704D0410804D014
:100BA00020F00104F7E722460EE0542000F09BF805
:100BB00007000ED0206D47F0010108435421206545
:100BC0003846FFF759FD3A4629463046BDE8F04120
:100BD0008CE70020D6E70000040100202DE9F04753
:100BE00004464FF000094FF0FF37C568D4E904868A
:100BF000A80707D0204600F055F9304602F074FAF5
:100C0000002802DA3846BDE8F087280502D54046BC
:100C1000FFF737FE4C212046FFF72EFD206D20F018
:100C2000010020654846EEE710B50446AFF30080AA
:100C30002046BDE81040FFF71FBB10B500F07CF95F
:100C4000BDE8104000F072B9004870470002002073
:100C5000004870470802002070477047704770478F
:100C600038B504460A4600206946AFF300800028E4
:100C700008BF38BD02460099204600F08DF90120DA
:100C800038BD012000F072B9F8B5AFF30080054619
:100C900000200C46102000BF0646A819A0420DD91E
:100CA000324669460020AFF30080070008BF00F01D
:100CB0005DF90098A04218BF0546C419FFF7C8FFA8
:100CC00005600746F01D20F007004619284600F091
:100CD0005CF9B44208BFF8BDA21B31463868BDE8D4
:100CE000F84000F059B970B50646FFF7B1FF056846
:100CF00006F10B0020F00704B4429CBF002070BD39
:100D00002B466A68BAB11068A04210D304F10801FA
:100D100088423CBF5068586007D351681019416041
:100D20001168091B016058601460101D70BD1346E6
:100D30005268002AE7D121462846FFF791FF002894
:100D4000DED170BD2DE9F041044616460D464769D7
:100D5000007B80072ED0384602F0D6F950BB3EB358
:100D6000012E02D0022E25D104E0204600F02EF9FB
:100D700005441DE0384602F0C3F9E168002841F05F
:100D80001001E16005DA204600F058F80120BDE8C6
:100D9000F081C9030BD56268E16A914200D811461F
:100DA000A26911442269891A814200DD084605447E
:100DB000002D01DA0220EAE7E16A6068E268814218
:100DC00006D29103E06203D522F4003141F0100213
:100DD000A6690027AE4213DCE16A814201D90B46C5
:100DE00000E0034603EB060C2369ACEB030CAC45B7
:100DF00006DD814201D98C4600E084469C4505D140
:100E0000A760276042F02000A5620DE0AD1BE669F7
:100E1000AE1B8142A66000D90846C01A281A20607D
:100E20005819606022F0200003490840E06000206B
:100E300084F84870ABE70000BFCFD7FFC16821F44A
:100E4000001141F08001C1600021816001607047A4
:100E50002DE9F047814614460E464FF0FF383248E0
:100E6000D5685769054209D03846A16902F084F96E
:100E7000002811DB2C48C0430540E5602B46324674
:100E80004946384602F07CF9A16920F00042B21AC6
:100E900011440028A16103D02046FFF7CFFF404650
:100EA000BDE8F08770B504460569C06A616888428C
:100EB00000D80846E16821F42011E160C90312D589
:100EC000A84208D02246411B2846FFF7C1FF10B1B7
:100ED0004FF0FF3070BD0020E562C4E90150E068CA
:100EE00020F48030E060002070BD10B50446C0687A
:100EF00020F02000E060A16AA06988420DD0204661
:100F0000FFF7D0FFE06820F4405040F01000E060B0
:100F1000A06AA0612069E062606044F24001E0687C
:100F20008843E06010BD000010000200002801D0DE
:100F300000F024B87047000010B5014602A000F090
:100F400066F8012010BD00005349475254524544F1
:100F50003A2052656469726563743A2063616E2752
:100F600074206F70656E3A200000000010B500F02C
:100F700067F8BDE81040FFF7D9BF0000014918200D
:100F8000ABBEFEE726000200704700210160C0E909
:100F90000110704710207047034640688C460028B7
:100FA00018BF88423CBF03464068F8D3186818440D
:100FB000884207D00CF1030020F00700001D411A01
:100FC000521A0146081D0A60FFF75BBC10B50146C6
:100FD000C268900703D0900607D5886A0AE000F03F
:100FE0005FF801210160881E10BD8B6948681844B4
:100FF0000B69C01A91F848301BB191F84910401A9A
:1010000010BD1103FCD50028FADD401E10BD70B5DF
:1010100005460C460A2000E06D1C00F039F835B199
:1010200028780028F8D102E0641C00F031F814B1EF
:1010300020780028F8D1BDE870400A2000F028B8D8
:1010400010B5012805D0002103A0FFF7E0FF012023
:1010500010BD09A1F8E7000053494752544D454DD2
:101060003A204F7574206F662068656170206D6549
:101070006D6F7279000000003A2048656170206D44
:10108000656D6F727920636F72727570746564003C
:1010900008B569468DF800000320ABBE08BD00000E
:1010A0000048704700020020FEE70000000000003A
:1010B00040F25840C2F2000000F022B800000000E8
:1010C0007047000000000000EFF3108072B600BF10
:1010D000FEE700000000000090F83510022909D159
:1010E000052180F835100068016821F001010160D8
:1010F00000207047802141650120704700000000FA
:10110000F0B581B00021009140F20C010446C2F21A
:10111000000148F2B513D0E916600A68C1F64E33F3
:10112000082137688140A2FB032539420CD0226890
:1011300013685B0708D5136823F004031360B160DC
:10114000616D41F00101616501218140394208D0A2
:1011500022685269120604D5B160616D41F0020146
:10116000616504218140394208D0226812689207E3
:1011700004D5B160616D41F00401616510218140C9
:10118000394215D020680268120711D5B160016894
:101190004903016806D4C90506D4016821F0080195
:1011A000016001E0080342D4216C09B12046884760
:1011B000E16D202000FA01F23A4244D02068036831
:1011C000DB0640D5B26094F83520052A02681ED1AE
:1011D00022F016020260426922F080024261226C13
:1011E0000AB9A26C1AB1026822F0080202603F201C
:1011F0008840B060012084F83500216D002000296E
:1012000084F8340057D02046884701B0F0BD510320
:10121000016810D4C90512D4016821F010010160E1
:10122000012084F83500002084F8340007E0A16C28
:101230000029BBD1BCE7080301D4616C00E0E16B7D
:1012400009B120468847606DA8B3606DC0072ED0F5
:10125000052084F835002068A90A026822F00102FE
:101260000260009A013200928A421AD80268D207BC
:1012700017D0009A013200928A4212D80268D2072F
:101280000FD0009A013200928A420AD80268D2072F
:1012900007D0009A013200928A4202D80268D2072F
:1012A000DFD1012084F83500002084F83400E16C9F
:1012B00009B12046884701B0F0BD000000000000E1
:1012C000F0B581B0044600F0DBF9002C4DD00546A6
:1012D000022084F835000020216884F83400086872
:1012E00020F00100086000BF0868C00706D000F0C9
:1012F000C7F9401B052863D82168F5E748F23F028B
:10130000251D0868CFF2100200EA020620692CCDE4
:10131000324366691A43A7692A43E3691043256A81
:101320003043626A3843042A40EA030040EA050376
:101330001ED1D4E90A5E206B4EEA03021043086016
:101340004869BEF1000F20F0030040EA050040F0BC
:10135000040C13D0B7F5005F36D0002F43D1022D17
:1013600044D0012D39D04DB940E0012001B0F0BD8D
:101370000B60486920F0070040EA020C6FF00F0094
:101380004AF6AB2250FA81F0CAF6AA22A0FB022349
:1013900040F2FF32C1F814C0914343F251421B099D
:1013A000C0F600025F2888BF0431D05C3F22A165EF
:1013B0000023E06502FA00F08860012200201CE0B2
:1013C00003222023032018E0032DD7D80122402335
:1013D0000120DFE805F0120B1202AEF1C070B0FA86
:1013E00080F0400904E0032D04D3C7D1CEF30060A0
:1013F0000028C3D0012240230120636584F83520F2
:1014000001B0F0BD0000000070B590F834C0BCF130
:10141000010F4BD04FF0010C80F834C0D0F858E0E9
:1014200090F835C0BCF1010F3DD14FF0020C80F8AF
:1014300035C04FF0000CC0F854C0D0F800C084682C
:10144000056CC06DDCF80060402C26F48026CCF8DA
:101450000060CCF804300B4604BF13460A463F2117
:10146000CCF8083001FA00F0CCF80C20CEF80800D7
:10147000DCF8000040F01600CCF80000DCF81400A6
:1014800040F08000CCF814002DB1DCF8000040F0F2
:101490000800CCF80000DCF8000040F00100CCF8B7
:1014A0000000002070BD002180F83410022070BDC3
:1014B0002DE9F04F82B000F13E420A2302F1FF779E
:1014C00042F20042C4F2020243F6004E90424FEA5A
:1014D000B72208BF0923092AC4F2010E38BF4FEA18
:1014E000B72300244FF0010A00270026009306E0EE
:1014F00002370136202F04F1040400F0B5800AFA07
:1015000006F80B6813EA080FF2D0D1F8049009F03E
:10151000030AAAF10103012B16D80322836802FAF9
:1015200007F5CA68AB43BA401A438260C9F3001397
:1015300042684FEA460C6FEA050B22EA0802B34004
:101540001A4342600EE000BF0322BAF1030F02FA11
:1015500007F2BC466FEA020B04D1BC464FF0030A07
:1015600023E000BFC2688B6802EA0B0203FA0CF3A7
:10157000BAF1020F42EA0302C26016D16FF0030211
:1015800004F01C0502EA56020F23024403FA05FA8E
:10159000D2F820900B6929EA0A09AB4043EA090313
:1015A0001362D1F8049009F0030A02680AFA0CF3F6
:1015B00002EA0B0219F4403F4FF0010A42EA03022B
:1015C000026095D043F644034FF60849C4F2020383
:1015D000CFF6FF790F251A6842F480421A601A6824
:1015E00026F0030302F4804201920EEB0302019BFA
:1015F00004F00C0352F809C09D402CEA050C009D34
:1016000005FA03F343EA0C0342F80930DEF808C098
:101610004B684CEA0805DA0258BF2CEA080543F685
:101620000C499A02C4F20109CEF80850D9F800C05A
:101630004CEA080558BF2CEA08059A03C9F800507F
:10164000DEF804C04CEA080558BF2CEA0805DB03A5
:10165000CEF80450DEF8002042EA080558BF22EA1E
:101660000805CEF8005043E702B0BDE8F08F000057
:10167000002A08BF090481617047000000000000D3
:1016800040F2A050C2F20000006870470000000065
:1016900040F2180040F2A051C2F20000C2F2000174
:1016A00000780A68104408607047000000000000DD
:1016B00080B5032000F08CF80F2000F005F800F052
:1016C0002BF8002080BD0000B0B540F2180140F2B8
:1016D0000C02C2F20001C2F200024FF47A73044617
:1016E00009781268B3FBF1F1B2FBF1F1084600F0A2
:1016F000D3FE0F2C4FF001050CD858B94FF0FF3036
:1017000000222146002500F033F840F21C00C2F20E
:10171000000004602846B0BD82B043F64000C4F229
:101720000200016841F080510160016801F08051C0
:1017300001910199416841F480414160406800F4A1
:1017400080400090009802B0704700000000000048
:10175000002848BF70474EF2001300F01F014009F7
:10176000CEF20003012202FA01F143F82010704783
:1017700070B54EF60C5C4FF0FF36CEF2000C00F167
:101780006045DCF80030C3F3022E8EF00703042B13
:1017900028BF0423BEF1030406FA03F321EA030180
:1017A00000F00F0338BF0024043BB0F1FF3F634457
:1017B00006FA04F003F10C0301FA04F1C8BF05F5C1
:1017C000644322EA000008430001187070BD000065
:1017D0004EF60C514FF6FF03CEF200010A681A4094
:1017E00060F30A2242F0806040F0FD7008607047AC
:1017F000B0B582B043F6400047F20005C4F20200E3
:10180000C4F20005016841F080510160006800F0F9
:10181000805001900198286840F480302860FFF7DC
:101820002FFF04466868C00306D4FFF729FF001B9A
:10183000B0F57A7FF6D910E0286840F400302860CF
:10184000FFF71EFF044600BF6868800308D4FFF757
:1018500017FF001BB0F57A7FF6D9032002B0B0BDA8
:10186000002002B0B0BD00002DE9F041002800F0DA
:10187000C48043F608080446C4F202080D46D8F8AE
:10188000F80300F00F0088420DD2D8F8F80320F0DA
:101890000F002843C8F8F803D8F8F80300F00F0049
:1018A000A84240F0AA802068810717D5410705D5D6
:1018B000D8F8001041F4E051C8F80010010705D530
:1018C000D8F8001041F46041C8F80010D8F80010B2
:1018D000A26821F0F0011143C8F80010C00735D10B
:1018E000D8F8F80300F00F00A8420CD9D8F8F80394
:1018F00020F00F002843C8F8F803D8F8F80300F0E8
:101900000F00A84279D12068410707D5D8F8001008
:10191000E26821F4E0511143C8F80010000708D52F
:10192000D8F80000216920F4604040EAC100C8F8FE
:101930000000D8F8000000F00C00082812D004289D
:1019400033D147F64000C0F27D1032E060680228D3
:1019500048D001284DD158F8081C890350D40120E3
:10196000BDE8F08158F8042C58F8040C400247F602
:10197000400058F8041CC0F27D105CBF42F20040E9
:10198000C0F2F400C1F3881102F03F02A0FB010194
:101990000023FEF7B1FC58F8041C0222C1F30141F8
:1019A00002EB4101B0FBF1F003E042F20040C0F273
:1019B000F400D8F8001043F22A42C0F60002C1F346
:1019C0000311515C40F21C02C2F20002C84040F216
:1019D0000C01C2F2000108601068FFF775FE0020DC
:1019E000BDE8F08158F8081C890109D40120BDE840
:1019F000F08158F8081C890702D40120BDE8F08165
:101A0000D8F8001021F003010843C8F80000FFF7E0
:101A100037FE064641F28837D8F80000616800F0CA
:101A20000C00B0EB810F3FF45BAFFFF729FE801B8A
:101A3000B842F1D90320BDE8F081000000000000A9
:101A40002DE9F04182B0002869D00446007843F6C1
:101A50000006C007C4F202060BD0B06800F00C000C
:101A6000042840F098803068800302D56068002820
:101A700055D0207880071AD5B06810F00C0F09D027
:101A8000B06800F00C00082840F0A28070684002A6
:101A900000F19E803068800702D5E06801283ED1C1
:101AA0003068216920F0F80040EAC10030602078F9
:101AB000000738D42078400749D4A5695DB3B068E1
:101AC00000F00C00082840F0B780012D706826D087
:101AD00000F48001E269914221D100F03F01226AC5
:101AE00091421CD147F6C071626A0140B1EB821F7E
:101AF00015D1A16A0022CFF6FF7200F4403302EB49
:101B0000C1316FF30F018B4209D1E16A00F07060BF
:101B1000B0EB016F03D1002002B0BDE8F0810120DD
:101B200002B0BDE8F08160690028706F73D040F0AA
:101B300001007067FFF7A4FD054600BF706F8007C6
:101B4000B8D4FFF79DFD401B0228F7D90DE1306C9A
:101B500010F0805808D1306C40F080503064306C08
:101B600000F080500190019847F20007C4F200078E
:101B70003868C00540D4386840F480703860FFF79A
:101B80007FFD05463868C00536D4FFF779FD401B58
:101B90006428F7D9E9E0B06800F00C00082803D108
:101BA000706840023FF55FAF6068002800F0B080C9
:101BB000B0F5A02F00F0C480B0F5803F00F0C480E5
:101BC000306820F480303060306820F48020BEE03F
:101BD000E0680028306851D040F001003060FFF725
:101BE0004FFD0546306880073FF55AAFFFF748FDC7
:101BF000401B0228F6D9B8E0A068002850D005287C
:101C000067D0012869D0306F20F001003067306F55
:101C100020F0040064E020F001007067FFF730FD61
:101C2000054600BF706F80077FF544AFFFF728FDC2
:101C3000401B0228F6D998E0306820F080703060B0
:101C4000FFF71EFD022D05460CD100BF3068800154
:101C500040F18F80FFF714FD401B02284FF0030076
:101C6000F4D959E7306880017FF555AFFFF708FDDB
:101C7000401B02284FF00300F4D94DE720F001008B
:101C80003060FFF7FDFC0546306880077FF50FAF39
:101C9000FFF7F6FC401B02284FF00300F4D93BE7A6
:101CA000306F20F001003067306F20F004003067A3
:101CB000FFF7E6FC054641F2883700BF306F80072A
:101CC0001DD5FFF7DDFC401BB8424FF00300F5D9EE
:101CD00022E7306F40F004003067306F40F00100C1
:101CE0003067FFF7CDFC054641F28837306F80073B
:101CF00005D4FFF7C5FC401BB842F7D935E0B8F171
:101D0000000F7FF4DAAE306C20F080503064D4E6FF
:101D1000306820F480303060306820F480203060FB
:101D2000FFF7AEFC054600BF306880037FF5A1AE2B
:101D3000FFF7A6FC401B64284FF00300F4D9EBE644
:101D4000306840F480203060306840F4803030608B
:101D5000FFF796FC054600BF306880033FF589AE6B
:101D6000FFF78EFC401B6428F6D9032002B0BDE8C3
:101D7000F08104F11C070025CFF6FF758FCF0843D3
:101D8000002105EBC333CDF6FF7140EA8210194004
:101D900040EA0760084340F000507060306840F04F
:101DA00080703060FFF76CFC044600BF3068800133
:101DB0003FF5B1AEFFF764FC001B02284FF00300B3
:101DC000F4D9A9E600000000704700000000000000
:101DD0007047000000000000B0B582B00446006803
:101DE000416882684B0602F0400305D512F00105F8
:101DF00002D00BB9E16C05E00D0608D512F0020522
:101E000005D0216D204602B0BDE8B04008478D06E0
:101E10000ED512F4B0750BD0BBB194F85D30032B26
:101E200008D100210191C168019180680190019859
:101E300002B0B0BD236E43F0040323660023019378
:101E4000C368019383680193019B12F0200302F49D
:101E500080720CD0236E43F00103236600230193AC
:101E600083680193036823F040030360019B42B140
:101E7000226E42F0080222660022019282680192DC
:101E8000019A226E002AD3D04268890722F0E0022C
:101E900042604FF0010184F85D101FD0416842F6A6
:101EA000493521F003014160A06DC0F6000538B14D
:101EB0000565FFF711F918B1206E40F0400020666B
:101EC000606D0028B4D00565FFF706F90028AFD093
:101ED000206E40F04000206602B0B0BDE16F91E797
:101EE00040B1B0B50446406A30B10020206104F131
:101EF000140007E0012070476068B0F5827F03D0CE
:101F000004F11C00002101600025A56294F85D0029
:101F1000A8BB42F2794042F2A911C0F60000C0F617
:101F20000001606642F2B110A16642F2914142F2B4
:101F3000894242F28143C0F60000C0F60001C4E9C4
:101F40001D01D4F88410C0F60002C0F60003E2665A
:101F500041F6D152236741F6C95384F85C50C0F66C
:101F60000002C0F60003E267C4F8803029B942F2EB
:101F70002901C0F60001C4F88410204688470220D9
:101F800084F85D002068D4F80CE0BEF5E06F4EF4F4
:101F90000063026898BF0125B3F5706F22F040021C
:101FA0004FEA053C026001D00023A362D4E9013569
:101FB000D4E9042103F4827305F404452B4402F0B0
:101FC00002021A4401F001011144A26902F40073F3
:101FD000E569194405F038031944236A03F08003C6
:101FE000A56A194405F4005319430423016003EA68
:101FF00012410EF47063626A43EA0C0302F01002AD
:10200000656B194305F00803114319434160C16929
:1020100021F40061C16100202066012184F85D1077
:10202000B0BD0000000000002DE9F04F85B043F680
:1020300000050446C4F200050068A84202D005B0BD
:10204000BDE8F08F43F63006E846C4F2020641468A
:102050004FF00209002730694FF0030A40F4804036
:10206000306130694FF0050B00F48040009000981B
:10207000306840F480703060306800F48070009008
:102080000098306840F002003060306800F00200D4
:102090000090009805F5F430CDE900990297CDF84D
:1020A0000CA0CDF810B0FFF703FA4FF40040414602
:1020B000CDE9000902A880E8800C05F5E630FFF7BD
:1020C000F7F940F2584506F52150C2F20005C5E97E
:1020D00000074020C5E902074FF48060C5E9040706
:1020E0002846C5E90677C5E90877FFF7E9F808B19A
:1020F000FEF7EAFF2420002100226565AC63FFF7AC
:1021000037FB2420FFF724FB05B0BDE8F08F00006B
:102110002AB190F85C30012B07D102207047016E84
:1021200041F0800101660120704790F85D30012B7D
:102130000BD109290CD8DFE801F0051D2023262941
:102140002C2F15194266002129E090F85D302BB143
:10215000016E41F080010166012120E0092905D0CE
:102160000829F5D1C0F88420002118E0C0F88820A3
:10217000002114E08266002111E0C26600210EE019
:10218000026700210BE04267002108E0826700211E
:1021900005E0C267002102E0C0F880200021002293
:1021A00080F85C200846704770470000000000007F
:1021B00070470000000000002DE9F04381B00446A4
:1021C00090F85C00012803D1022001B0BDE8F08343
:1021D0001D4616460F464FF0010984F85C90FFF744
:1021E0004FFA94F85D1001295DD180460120002F3F
:1021F00018BF002E00F0B080032084F85D0000209E
:102200002066A763A687E6872064A4F84400A4F8A4
:102210004600A168B1F5004FC4E91300206807D15A
:10222000016821F040010160016841F480410160D2
:102230000168490603D4016841F04001016061680A
:10224000731EB1FA81F1E268B3FA83F349095B09BD
:10225000B2F5E06F41EA030127D931B137F8021B2B
:10226000C160A763E18F0139E187E18F00295CD06C
:102270006E1C00BF8168890708D4FFF701FA6EB1B0
:10228000A0EB0800A84209D36EE000BFA16B31F8B3
:10229000022BC260A163E08F0138E087E08F002845
:1022A00043D02068E6E7022056E000294FF6FE7191
:1022B00011D0E28F022A05D337F8022BC2604FF605
:1022C000FE7004E03A780273A06B471C481CA763B9
:1022D000E28F1044E087E08F38B36E1C4F1C0BE098
:1022E000A16B09780173A06B0130A0633846E18FC0
:1022F0000844E087E08FC0B120688168890709D46D
:10230000FFF7BEF9002EF5D0A0EB0800A842F1D3EC
:102310002CE000BFE18F0229E2D3A16B31F8022B40
:10232000C2604FF6FE70A163E1E7204629464246AF
:1023300000F05EFC00281CBF20202066A06838B991
:10234000002000902068C16800918068009000988B
:10235000206E002818BF012084F85D90002184F8C9
:102360005C1001B0BDE8F0830320F5E70320F3E73C
:10237000B0B5044690F85C00012801D10220B0BD40
:10238000012084F85C0094F85D00012847D1012009
:10239000002918BF002A43D0032084F85D000025DF
:1023A0002566A163A287E2872564C4E91355A4F8D2
:1023B0004450A4F84650A068B0F5004F226807D1F9
:1023C000106820F040001060106840F480401060F9
:1023D000606D42F6813C42F6793E42F65933C0F6D2
:1023E000000CC0F6000EC0E90FCEC0F60003C364B7
:1023F000E36805655568B3F5E06F25F480435360E5
:102400001AD88369B3F5005F16D1E38FDB075368F1
:102410000AD123F480435360E38F5B080BE0022072
:10242000002184F85C10B0BD43F480435360E38F17
:10243000012505EB5303E387E38F0C32FEF7E4FF3E
:1024400038B1206E40F010002066012084F85D0055
:10245000E6E720680168490603D4016841F04001BD
:102460000160416841F020014160416841F0020192
:1024700041600020D4E70000704700000000000029
:1024800070470000000000007047000000000000DE
:102490007047000000000000411E0020B0EB116FEB
:1024A00001D0012070474EF21002F023CEF200025C
:1024B00051604EF62351CEF200010B70072190605F
:1024C0001160704700000000FEE7000000000000FF
:1024D00080B582B043F630000022C4F202000168E9
:1024E00041F4001101600068002100F40010019027
:1024F00001980F20FFF73CF90F2002B0BDE88040A3
:10250000FFF726B9000000002DE9F04387B043F63D
:1025100030004FF00009C4F20200CDF8189040F2EC
:10252000004500220168C4F2020541F00201016089
:10253000016801F0020101910199016841F4807183
:102540000160016801F4807101910199016841F015
:102550002001016000684FF4407100F020000190FC
:1025600001982846FFF784F805F5805440210022A1
:1025700020464FF04008FFF77BF802AE4FF4807022
:102580000290284631460127CDE90377CDF8149013
:10259000FEF78EFF4FF400703146CDE902070220AE
:1025A000CDE904092846FEF783FF20463146CDE9F0
:1025B0000287CDE90479FEF77BFF07B0BDE8F08321
:1025C00080B540F2B84043F60001C2F20000C4F208
:1025D00000014FF4E06201604FF48271416000211C
:1025E0008160C0E9032141614FF4007282611822C9
:1025F000C0E90721C0E909110722C0E90B21082120
:102600004163FFF76DFC002808BF80BDBDE8804036
:10261000FEF75ABD00000000FEE7000000000000C9
:10262000FEE70000000000002DE9F047532898BFA6
:102630002F2903D8532A98BF2F2B01D9BDE8F08743
:10264000DDF820C0904288BF994209D8904238BF37
:10265000994205D3904240F281808646104684E03C
:10266000904202D91F46864603E00F469646194619
:102670000246AEEB0200CB1B984237DD9645DDD318
:1026800040F214091B014FF00108C2F200094FF09B
:10269000540A174609E000BFD9F80040A65C35434C
:1026A000A55401373AB29645C8DBFCB2532CF8D892
:1026B000AEEB02025A4392FBF0F20832D51702EB5E
:1026C0001572A1EB1215EAB22F2AEAD8D20805F04A
:1026D000070512FB0A42BCF1000F08FA05F5DBD131
:1026E000D9F80040A65C26EA0505D9E7B942A5D38A
:1026F00040F2140900014FF00108C2F200094FF046
:10270000540A3E4609E000BFD9F80050AF5C3C4394
:10271000AC54013637B2B94290DBF2B22F2AF8D866
:10272000CC1B444394FBF3F40834E71704EB177411
:10273000AEEB1414E7B2532FEBD802F00704D20823
:1027400012FB0A72BCF1000F08FA04F4DCD1D9F8CC
:102750000070BD5C25EA0404BC54DAE70F469942D8
:1027600084BF1F460B4696463946AEEB00025C1A04
:10277000A24238DD8645FFF461AF40F2140923011F
:102780004FF00108C2F200094FF0540A074609E071
:10279000D9F80040265C35432554013738B28645C8
:1027A000FFF64CAFFCB2532CF7D8AEEB0000584309
:1027B00090FBF2F00830C51700EB157001EB101517
:1027C000E8B22F28E9D8C00805F0070510FB0A4039
:1027D000BCF1000F08FA05F5DAD1D9F80040265C03
:1027E00026EA0505D8E78B4217D101F0070201233D
:1027F00003FA02F25423C908BCF1000F11FB0300D5
:1028000040F21401C2F2000109680B5C0CBF23EA1C
:1028100002021A430A54BDE8F08738BFBDE8F087CA
:1028200040F214084FEA021A4FF0010EC2F20008FB
:102830004FF054090F460CE0EA0812FB0911D8F8D2
:102840000020555C35435554013739B28B42FFF6B1
:10285000F5AEFDB22F2DF7D8591A0AFB01F191FB05
:10286000F4F10831CE1701EB167100EB1111C9B26A
:102870005329E9D805F00706BCF1000F0EFA06F659
:10288000DAD1ED0815FB0911D8F800506A5CB243A3
:102890006A54D9E700000000F0B581B040F200446E
:1028A00006460820C4F2020460F3DF018DF802102E
:1028B0004FF4007100222046FEF7DAFE04F5805541
:1028C000402100222846FEF7D3FE40F2B8470DF122
:1028D0000201C2F2000701220A233846FFF76CFC0E
:1028E000402101222846FEF7C3FE4FF40071012269
:1028F0002046FEF7BDFE46F080008DF803004FF441
:10290000007100222046FEF7B3FE40210022284637
:10291000FEF7AEFE0DF1030101220A233846FFF750
:102920004BFC402101222846FEF7A2FE4FF4007125
:1029300001222046FEF79CFE01B0F0BD0000000021
:1029400070B582B040F200444FF48071C4F20204CA
:1029500001222046FEF78CFE04F58055402101221D
:102960002846FEF785FE21208DF801004FF4007106
:1029700000222046FEF77CFE402100222846FEF77A
:1029800077FE40F2B8460DF10101C2F200060122C5
:102990000A233046FFF710FC402101222846FEF7AB
:1029A00067FE4FF4007101222046FEF761FEBE2053
:1029B0008DF802004FF4007100222046FEF758FE09
:1029C000402100222846FEF753FE0DF102010122AC
:1029D0000A233046FFF7F0FB402101222846FEF78C
:1029E00047FE4FF4007101222046FEF741FE1320FE
:1029F0008DF803004FF4007100222046FEF738FEE8
:102A0000402100222846FEF733FE0DF1030101228A
:102A10000A233046FFF7D0FB402101222846FEF76B
:102A200027FE4FF4007101222046FEF721FE2020F0
:102A30008DF804004FF4007100222046FEF718FEC6
:102A4000402100222846FEF713FE01A901220A2395
:102A50003046FFF7B1FB402101222846FEF708FE71
:102A60004FF4007101222046FEF702FE09208DF886
:102A700005004FF4007100222046FEF7F9FD4021C9
:102A800000222846FEF7F4FD0DF1050101220A237C
:102A90003046FFF791FB402101222846FEF7E8FD72
:102AA0004FF4007101222046FEF7E2FD08208DF868
:102AB00006004FF4007100222046FEF7D9FD4021A8
:102AC00000222846FEF7D4FD0DF1060101220A235B
:102AD0003046FFF771FB402101222846FEF7C8FD72
:102AE0004FF4007101222046FEF7C2FD0C208DF844
:102AF00007004FF4007100222046FEF7B9FD402187
:102B000000222846FEF7B4FD0DF1070101220A2339
:102B10003046FFF751FB402101222846FEF7A8FD71
:102B20004FF4007101222046FEF7A2FD02B070BDF5
:102B3000704700000000000040F2B840C2F2000000
:102B4000FFF74AB900000000806B0021A0F8461092
:102B5000C187C16F08470000806B0168C26F4B6876
:102B600023F003034B60016E41F010010166012167
:102B700080F85D1010470000806B016F084700006F
:102B8000B0B582B00546846BFEF77AFD2968096806
:102B9000C90525D402462068416821F02001416022
:102BA000416821F0020141606421204600F020F8D4
:102BB00018B1206E40F020002066A06838B90020CF
:102BC00001902068C16801918068019001980020FF
:102BD000E087012084F85D00206E08B1E16F00E01D
:102BE000616E204602B0BDE8B0400847000000001A
:102BF00070B582B015460E464FF4C05132462B4692
:102C0000044600F059F808BB40F20C0049F6817107
:102C1000C2F20000C1F25E610068A0FB0101480D34
:102C20004FF47A71484301906068B0F5827F15D106
:102C3000204631462A4600F0B7F838B94FF4C06153
:102C4000204632462B4600F037F880B3206E40F025
:102C500020002066032002B070BD00BF019800284C
:102C6000ECD0019801380190206880680006E5D515
:102C700001980028E2D0019801380190206880680E
:102C80000006DBD501980028D8D0019801380190C2
:102C9000206880680006D1D501980028CED0019820
:102CA00001380190206880680006D7D4C6E700206C
:102CB00002B070BD000000002DE9F04F83B01E4649
:102CC00090460D4682464FF000098DF80790FEF7BA
:102CD000D7FC301A00EB0807FEF7D2FC40F20C01DB
:102CE0002322C2F20001DAF800B009685143090D4D
:102CF00079430291DBF8081029424FD0064608F1CB
:102D00000104584603E000BF816829421AD0B5F596
:102D1000C06F05D19BF80C108DF807109DF80710B7
:102D2000002CF1D0FEF7ACFC801BB8420DD202980B
:102D300002990028A1F10101029108BF0746DAF8C3
:102D40000000E1E74FF0000928E0DAE90001B1F501
:102D5000827F426822F0E00141600AD1DAF808106F
:102D6000B1F5004F11BFB1F5806F016821F040014E
:102D70000160DAF82810B1F5005F07D1016821F48D
:102D800000510160016841F40051016001208AF89E
:102D90005D0000208AF85C004FF00309484603B04C
:102DA000BDE8F08F00000000F0B581B015460E467A
:102DB0000446FEF765FC281A8719FEF761FC40F20D
:102DC0000C01C2F200010968C1F3CB3179430091D3
:102DD00021688A68120602D4002001B0F0BD0546C1
:102DE000013602E088680006F6D5002EFAD0FEF71C
:102DF00047FC401BB84209D2009800990028A1F175
:102E00000101009108BF07462168EBE7D4E9000102
:102E1000B1F5827F426822F0E001416009D1A168EA
:102E2000B1F5004F11BFB1F5806F016821F040018D
:102E30000160A16AB1F5005F07D1016821F400517A
:102E40000160016841F400510160012084F85D00D7
:102E5000002084F85C00032001B0F0BD00000000F9
:102E600070470000000000002DE9F04F81B040F2F3
:102E70009C584CF6CD41C2F20008CCF6CC4140F251
:102E8000485740F29859D8F80000C2F200070130C4
:102E9000C2F20009A0FB011240F2010AC8F2000AC6
:102EA000110901EB8101A0EB8106C9F8006007EB75
:102EB000860317F826000026009659789A78DB7862
:102EC000FFF7B2FBD8F800000125009507EB80035F
:102ED00017F8200059789A78DB78FFF7A5FB40F2C5
:102EE000100BD8F80000C2F2000BD9F800609BF973
:102EF000004057F8200047F8260021183046CAB293
:102F0000542A14D3FDF7BEF95146002CCCBF4FF024
:102F1000FF356FF0004100EB400090FBF1F017F837
:102F2000261028448BF800000144D9F8000007EB74
:102F300080059BF9024007F8261015F8022F22445D
:102F4000D3B2542B16D3FDF79DF95146002CD8BFB0
:102F50006FF000414FF0010200EB4000C8BF4FF09E
:102F6000FF3290FBF1F0297810448BF802000A1828
:102F7000D9F8000007EB80069BF901402A7016F88B
:102F8000011F2144CBB2302B14D3FDF77BF95146FE
:102F9000002CD8BF6FF000414FF00102C8BF4FF0C6
:102FA000FF3290FBF1F0317810448BF801000144BE
:102FB000D9F8000007EB80059BF90340317015F844
:102FC000032F2244D3B2302B13D3FDF75BF9002C2F
:102FD0004FF00101D8BF6FF0004AC8BF4FF0FF317A
:102FE00090FBFAF02A7808448BF803000244D9F8E1
:102FF00000002A70C8F8000001B0BDE8F08F0000A2
:10300000FEF746BB0000000080B592B043F64001D9
:103010000020C4F202010B90CDE90900CDE90700C0
:103020000590CDE90300CDE901000A6842F0805225
:103030000A60096801F08051009147F20001009A8E
:10304000C4F200010A6842F440420A6009680122A1
:1030500001F44041009100990221CDE90C100820B3
:103060000E90D8200691CDE90F0106A809921022F2
:103070000A921191FEF7E4FC18B1EFF3108072B6DA
:10308000FEE7FEF7B5FB20B1EFF3108072B600BF8C
:10309000FEE70F20019002200290002003904FF4E1
:1030A000A05004904FF48050059001A80721FEF72E
:1030B000DBFB20B1EFF3108072B600BFFEE712B069
:1030C00080BD0000000000004EF68850CEF20000E7
:1030D000016841F4700101607047000000000000C9
:1030E000FEE700000000000048F20101411A002044
:1030F000022988BF4FF0FF30704700000000000039
:10310000002070470000000048F20101411A002031
:10311000032938BF0120704710B510B3044600786A
:103120003A281ED143F242412046C0F60001FDF785
:10313000F7F9C8B143F249412046C0F60001FDF756
:10314000EFF9A0B143F23A412046C0F60001FDF785
:10315000E7F94FF0FF31002808BF48F203010846A5
:1031600010BD4FF0FF3010BD48F2010010BD48F215
:10317000020010BD000000004FF0FF30704700005B
:1031800048F20303984229D048F20203984227D11B
:1031900022B380B540F6006C4FF06043CEF2000CD5
:1031A00004E000BF83F800E0013A1CD011F801EB05
:1031B000DCF88000C0071CBFDCF800005FEAC070CC
:1031C000F2D000BF1868002801BF186800281868EE
:1031D0000028E7D118680028F4D0E3E70020704702
:1031E0004FF0FF307047002080BD0000000000005D
:1031F00084B04EF66074CEF20004FEF759FAFFF781
:1032000003FFFFF781F9FFF763F9FFF7D9F9FFF73C
:1032100097FBFEF735FABFF34F8FBFF36F8F002197
:1032200044F8101C4FF6B4530127BFF34F8FCFF66D
:10323000FF730546BFF36F8FE25843F6E07B42F41D
:103240000032E2504FF62462CFF6FF72BFF34F8F89
:10325000BFF36F8FA1504FF62061CFF6FF71BFF320
:103260004F8F6158CB08C1F34E32C1F3C90C07EB45
:10327000D101ACF101079807ACF1020A01F0030695
:10328000BB0703934FEA8A710291ACF103010191EC
:1032900004E000BF002AA2F101022BD00BEA421188
:1032A00063468EB1012E40EA010323603B460BD0FA
:1032B000039B022E43EA01032360534604D0029B82
:1032C0000B432360019B00BFBCF1030FE2D341EA33
:1032D0008371013301F1404881F0004901F1804ED2
:1032E000043B2160C4F80080C4F80090C4F800E0FA
:1032F000F6D1CFE74FF6B45141F2004BCFF6FF7154
:10330000C4F2020BBFF34F8F6058002240F48030AC
:103310006050BFF34F8FBFF36F8F40215846FEF7C9
:10332000A7F940F2B84443F2E932C2F20004C0F611
:10333000000200212046FEF7EBFE40210122584604
:10334000FEF796F900200021FFF7A6FA402100229F
:103350005846FEF78DF943F25C4040F2602AC0F611
:103360000000C2F2000A5146A146006887B220461A
:103370003A46FEF7FDFF40F244580026C2F200082C
:1033800002E000BFFFF770FDD8F80000B0B10020E8
:10339000C8F800004021012258460136FEF768F9BE
:1033A00000200021FFF778FA402100225846FEF75E
:1033B0005FF9484651463A46FEF7DAFFFEF760F9F4
:1033C0000446401BB0F57A7FDCD903A03146FDF7F7
:1033D0000BF800262546D5E74650533A2025640DC4
:1033E0000A0000000000000040F244500121C2F237
:1033F0000000016070478A68002A01DCFDF768BAA6
:10340000521E8A604A68C0B2531C4B6010707047ED
:10341000F1EE100A4FF6FF71C0F2C03120EA010050
:1034200040F04070E1EE100A70470000000000001C
:10343000000001020304060708093A5354444552A8
:1034400052003A535444494E003A5354444F555451
:10345000000006101600061016000000F80100001B
:103460008034000800000020200000000402000852
:10347000A034000820000020880B00002002000873
:103480000000000000000000000000000024F40024
:10349000010203046002002001000000100000008F
:04000005080001C925
:00000001FF
